:100000000C9435000C9450020C947D020C945D000D
:100010000C945D000C945D000C945D000C945D00EC
:100020000C945D000C945D000C945D000C945D00DC
:100030000C945D000C945D000C945D000C945D00CC
:100040000C94AA020C945D000C94C5030C945D0002
:100050000C945D000C945D000C945D000C945D00AC
:100060000C945D000C945D002C0111241FBECFEF99
:10007000D4E0DEBFCDBF11E0A0E0B1E0ECEDF8E0F0
:1000800002C005900D92AA33B107D9F711E0AAE397
:10009000B1E001C01D92A03DB107E1F710E0CAE652
:1000A000D0E004C02297FE010E946804C836D10740
:1000B000C9F70E9425010C946C040C940000CF92A7
:1000C000DF92EF92FF920F931F93DF93CF9300D0B5
:1000D00000D000D0CDB7DEB78AE391E00E943A01AC
:1000E000882309F49AC08AE391E00E9437018230A4
:1000F00009F093C0EE2410E000E06E010894C11CEA
:10010000D11C8AE391E00E943A018823D1F38AE36B
:1001100091E00E943701282F8D3009F47EC08A308B
:1001200009F47BC0833009F478C0823009F475C0CB
:1001300080538A3010F4282F05C0822F81548630D6
:1001400008F42753812F90E010FD02C0022F0DC04C
:1001500095958795302F3295307F322BF601E80F39
:10016000F91F3083059709F0E3261F5F1C3048F222
:100170001C3009F052C060E071E08AE391E00E9417
:1001800042018E010F5F1F4F86E0C82ED12CCC0E8E
:10019000DD1EF801F080FFE0FF1530F06EE071E049
:1001A0008AE391E00E9442014F2D50E060E070E050
:1001B00020E130E08AE391E00E943B0260E171E0DF
:1001C0008AE391E00E9442010F5F1F4F0C151D054D
:1001D00001F78AE391E00E945A0162E171E08AE34B
:1001E00091E00E9442011E81412F50E060E070E0EA
:1001F00020E130E08AE391E00E943B021E1519F0F5
:100200006DE171E002C068E271E08AE391E00E9472
:1002100071018AE391E00E945A0126960FB6F89484
:10022000DEBF0FBECDBFCF91DF911F910F91FF9029
:10023000EF90DF90CF90089540E855E260E070E0E5
:100240008AE391E00E943D0108950E941A030E94F2
:100250001C010E945F00FDCF88E391E090933B0179
:1002600080933A010895862F0E948D0308950E947D
:10027000A60308950E9495030895CB01BA010E9438
:10028000540308950F931F93CF93DF938C01EB01D9
:1002900009C02196D801ED91FC910190F081E02DEB
:1002A000C801099568816623A1F7DF91CF911F915D
:1002B0000F9108950F931F938C01DC01ED91FC9138
:1002C0000190F081E02D6DE00995D801ED91FC9150
:1002D0000190F081E02D6AE0C80109951F910F910E
:1002E00008950F931F938C010E944201C8010E9440
:1002F0005A011F910F9108952F923F924F925F9252
:100300006F927F928F929F92AF92BF92CF92DF9225
:10031000EF92FF920F931F93DF93CF93CDB7DEB78A
:10032000A0970FB6F894DEBF0FBECDBF1C016A01C7
:100330007B01411551056105710549F4DC01ED9121
:10034000FC910190F081E02D60E3099554C0882470
:1003500099245401422E55246624772401E010E0AC
:100360000C0F1D1F080D191DC701B601A301920135
:100370000E941504F80160830894811C911CA11C43
:10038000B11CC701B601A30192010E941504C90165
:10039000DA016C017D01C114D104E104F104F1F62C
:1003A00081E0E82EF12CEC0EFD1EE80CF91C3E015C
:1003B0000894611C711CD501C4010197A109B10900
:1003C0006C01C818D90814C0F601EE0DFF1D60813C
:1003D0006A3010F4605D01C0695CD101ED91FC915F
:1003E0000190F081E02DC10109950894E108F10820
:1003F0006E147F0449F7A0960FB6F894DEBF0FBEC7
:10040000CDBFCF91DF911F910F91FF90EF90DF90C3
:10041000CF90BF90AF909F908F907F906F905F90A4
:100420004F903F902F900895EF92FF920F931F935C
:10043000CF93DF93EC017A018B0177FF0FC0E88146
:10044000F9810190F081E02D6DE2099510950095FC
:10045000F094E094E11CF11C011D111D2AE0B8018B
:10046000A701CE010E947C01DF91CF911F910F91D6
:10047000FF90EF900895DC012115310541F4ED91D5
:10048000FC910190F081E02D642F099508952A30A8
:10049000310519F40E94140208950E947C01089508
:1004A0001F920F920FB60F9211242F933F934F93E9
:1004B0005F936F937F938F939F93AF93BF93EF93CC
:1004C000FF9380913C0190913D01892B29F0E091AF
:1004D0003C01F0913D010995FF91EF91BF91AF91E2
:1004E0009F918F917F916F915F914F913F912F914C
:1004F0000F900FBE0F901F9018951F920F920FB67E
:100500000F9211242F933F934F935F936F937F9399
:100510008F939F93AF93BF93EF93FF9380913E018F
:1005200090913F01892B29F0E0913E01F0913F012C
:100530000995FF91EF91BF91AF919F918F917F911D
:100540006F915F914F913F912F910F900FBE0F9040
:100550001F9018951F920F920FB60F9211242F9390
:100560008F939F93AF93BF938091400190914101EE
:10057000A0914201B09143010196A11DB11D80934C
:10058000400190934101A0934201B09343018091B7
:10059000440190914501A0914601B09147018050DE
:1005A000904CAF4FBF4F8093440190934501A0936F
:1005B0004601B093470127C08091440190914501C5
:1005C000A0914601B091470180589E43A040B040A1
:1005D0008093440190934501A0934601B093470155
:1005E0008091480190914901A0914A01B0914B013D
:1005F0000196A11DB11D8093480190934901A093DC
:100600004A01B0934B018091440190914501A09122
:100610004601B091470181589E43A040B04060F62A
:10062000BF91AF919F918F912F910F900FBE0F901F
:100630001F901895789484B5826084BD84B58160DC
:1006400084BD85B5826085BD85B5816085BDEEE6DA
:10065000F0E0808181608083E1E8F0E08081826069
:100660008083808181608083E0E8F0E08081816028
:100670008083E1EBF0E0808184608083E0EBF0E058
:10068000808181608083EAE7F0E0808184608083FC
:1006900080818260808380818160808380818068A6
:1006A00080831092C1000895EF92FF920F931F93E1
:1006B0007B018C0122E030E040E050E00E943704F2
:1006C000205C3D4B404F5F4FCA01B901A801970123
:1006D0000E943704C901DA010197A109B109292F44
:1006E0003A2F4B2F552747FD5A950196A11DB11D55
:1006F0002093C50081508093C400E1ECF0E080813C
:10070000806180838081886080838081806880832D
:100710001F910F91FF90EF900895982F8091C00046
:1007200085FFFCCF9093C600089580914C01909175
:100730004D0180589F4F20914E0130914F01821BF7
:10074000930B60E870E00E940204089540914E010E
:1007500050914F0180914C0190914D018417950764
:1007600019F42FEF3FEF0FC0FA01E05BFE4F20813D
:10077000CA01019660E870E00E94020490934F0164
:1007800080934E0130E0C90108951F920F920FB679
:100790000F9211242F933F934F935F936F937F9307
:1007A0008F939F93AF93BF93EF93FF934091C600B6
:1007B000E0914C01F0914D01CF01019660E870E0AD
:1007C0000E9402049C0180914E0190914F012817D4
:1007D000390739F0E05BFE4F408330934D012093A1
:1007E0004C01FF91EF91BF91AF919F918F917F91BC
:1007F0006F915F914F913F912F910F900FBE0F908E
:100800001F90189597FB092E07260AD077FD04D074
:1008100049D006D000201AF4709561957F4F089555
:10082000F6F7909581959F4F0895A1E21A2EAA1B85
:10083000BB1BFD010DC0AA1FBB1FEE1FFF1FA21790
:10084000B307E407F50720F0A21BB30BE40BF50B8D
:10085000661F771F881F991F1A9469F76095709516
:10086000809590959B01AC01BD01CF01089597FB48
:10087000092E05260ED057FD04D0D7DF0AD0001C64
:1008800038F450954095309521953F4F4F4F5F4F2D
:100890000895F6F790958095709561957F4F8F4FED
:1008A0009F4F0895AA1BBB1B51E107C0AA1FBB1F86
:1008B000A617B70710F0A61BB70B881F991F5A95EC
:1008C000A9F780959095BC01CD010895EE0FFF1F0B
:0C08D0000590F491E02D0994F894FFCFFE
:1008DC00352D6279746520636F64653A20003000B1
:1008EC002000436865636B73756D3A2000202D2DD5
:1008FC00206572726F722E00202D2D207061737323
:0A090C0065642E00000000003301B6
:00000001FF
